:020000040800F2
:1000000000070020E50400080D1D00088D1C0008F5
:10001000E51C00088D1C0008B91C0008E704000856
:10002000E7040008E7040008E7040008C1430008EB
:10003000E7040008E7040008E7040008E7040008F4
:10004000E7040008E7040008E7040008E7040008E4
:10005000E7040008E70400085D540008895400081C
:10006000B5540008E15400080D550008E7040008E5
:10007000E7040008E7040008E7040008E7040008B4
:10008000E7040008E7040008E7040008C12B0008A3
:100090002D2C0008812C0008D52C000839550008AB
:1000A000E7040008E7040008E7040008E704000884
:1000B000D1520008E7040008E7040008E70400083C
:1000C000E7040008E7040008E7040008E704000864
:1000D000E7040008E7040008E7040008E704000854
:1000E000A1550008E7040008E7040008E704000839
:1000F000E7040008E7040008E7040008E704000834
:10010000E7040008E7040008E7040008E704000823
:10011000E7040008E7040008E7040008E704000813
:10012000E7040008E7040008E7040008E704000803
:10013000E7040008E7040008E7040008E7040008F3
:10014000E7040008E7040008E7040008F94A00088B
:10015000E7040008E7040008E7040008E7040008D3
:10016000E7040008E7040008E7040008E7040008C3
:10017000E7040008E7040008E7040008E7040008B3
:10018000E7040008E7040008E7040008E7040008A3
:10019000E7040008E7040008E7040008E704000893
:1001A000E7040008E7040008E7040008E704000883
:1001B000E7040008E7040008E7040008E704000873
:1001C000E7040008E7040008E7040008E704000863
:1001D000E7040008E7040008E7040008E704000853
:1001E00053B94AB9002908BF00281CBF4FF0FF319E
:1001F0004FF0FF3000F074B9ADF1080C6DE904CE9A
:1002000000F006F8DDF804E0DDE9022304B07047F1
:100210002DE9F047089D04468E46002B4DD18A42B9
:10022000944669D9B2FA82F252B101FA02F3C2F1EC
:10023000200120FA01F10CFA02FC41EA030E94407D
:100240004FEA1C48210CBEFBF8F61FFA8CF708FB9E
:1002500016E341EA034306FB07F199420AD91CEB76
:10026000030306F1FF3080F01F81994240F21C81A8
:10027000023E63445B1AA4B2B3FBF8F008FB1033F0
:1002800044EA034400FB07F7A7420AD91CEB040425
:1002900000F1FF3380F00A81A74240F207816444F5
:1002A000023840EA0640E41B00261DB1D44000237A
:1002B000C5E900433146BDE8F0878B4209D9002DDE
:1002C00000F0EF800026C5E9000130463146BDE868
:1002D000F087B3FA83F6002E4AD18B4202D38242D2
:1002E00000F2F980841A61EB030301209E46002D81
:1002F000E0D0C5E9004EDDE702B9FFDEB2FA82F2D6
:10030000002A40F09280A1EB0C014FEA1C471FFA33
:100310008CFE0126200CB1FBF7F307FB131140EA1A
:1003200001410EFB03F0884208D91CEB010103F1E7
:10033000FF3802D2884200F2CB804346091AA4B2A9
:10034000B1FBF7F007FB101144EA01440EFB00FE7D
:10035000A64508D91CEB040400F1FF3102D2A645E2
:1003600000F2BB800846A4EB0E0440EA03409CE781
:10037000C6F12007B34022FA07FC4CEA030C20FA2E
:1003800007F401FA06F31C43F9404FEA1C4900FA4E
:1003900006F3B1FBF9F8200C1FFA8CFE09FB1811CB
:1003A00040EA014108FB0EF0884202FA06F20BD93E
:1003B0001CEB010108F1FF3A80F08880884240F28E
:1003C0008580A8F102086144091AA4B2B1FBF9F0D2
:1003D00009FB101144EA014100FB0EFE8E4508D9CD
:1003E0001CEB010100F1FF346CD28E456AD9023852
:1003F000614440EA0840A0FB0294A1EB0E01A14237
:10040000C846A64656D353D05DB1B3EB080261EBA4
:100410000E0101FA07F722FA06F3F1401F43C5E97E
:10042000007100263146BDE8F087C2F12003D840B4
:100430000CFA02FC21FA03F3914001434FEA1C47F6
:100440001FFA8CFEB3FBF7F007FB10360B0C43EAE8
:10045000064300FB0EF69E4204FA02F408D91CEB98
:10046000030300F1FF382FD29E422DD90238634496
:100470009B1B89B2B3FBF7F607FB163341EA034136
:1004800006FB0EF38B4208D91CEB010106F1FF3885
:1004900016D28B4214D9023E6144C91A46EA00467C
:1004A00038E72E46284605E70646E3E61846F8E60E
:1004B0004B45A9D2B9EB020864EB0C0E0138A3E757
:1004C0004646EAE7204694E74046D1E7D0467BE738
:1004D000023B614432E7304609E76444023842E7B0
:1004E000704700BF02E000F000F8FEE772B63A483D
:1004F00080F30888394880F3098839484EF6085156
:10050000CEF20001086040F20000CCF200004EF68E
:100510003471CEF200010860BFF34F8FBFF36F8FCD
:1005200040F20000C0F2F0004EF68851CEF2000119
:100530000860BFF34F8FBFF36F8F4FF00000E1EE05
:10054000100A4EF63C71CEF200010860062080F3DE
:100550001488BFF36F8F03F0B3FF03F08FFF04F035
:100560001BFE4FF055301F491B4A91423CBF41F8DA
:10057000040BFAE71C49194A91423CBF41F8040BAD
:10058000FAE71A491A4A1B4B9A423EBF51F8040B2C
:1005900042F8040BF8E700201749184A91423CBF83
:1005A00041F8040BFAE703F06DFF04F049FE144C28
:1005B000144DAC4203DA54F8041B8847F9E700F005
:1005C00041F8114C114DAC4203DA54F8041B884732
:1005D000F9E703F055BF00000007002000230020CA
:1005E000000000080001002000070020005B000858
:1005F000002300205023002050230020144000201E
:10060000E0010008E0010008E0010008E001000846
:100610002DE9F04F2DED108AC1F80CD0C3689D462E
:10062000BDEC108ABDE8F08F002383F311882846C3
:10063000A047002003F06EFAFEE703F0E9F900DFBF
:10064000FEE70000F8B503F065FE074603F0B2FED2
:10065000044688BB1D4B9F422ED001339F422ED0B3
:100660001B4B27F0FF029A422CD1F8B200F01AFD82
:10067000264642F2107500F01FFF00F019FD08B980
:100680000646054634B1134B9F4203D003F08AFE61
:1006900000252E46002003F047FE0EB100F062F860
:1006A00001F0C6FA00F02AFF01F052F9284600F0E6
:1006B000B5F800F057F8F9E726460025DBE70546D0
:1006C0000126D8E7064641F28835D4E7010007B095
:1006D000000008B0263A09B008B501F00BF9A0F106
:1006E00020035842584108BD07B541F212030221C8
:1006F00001A8ADF8043001F01BF903B05DF804FB6C
:1007000010B5202383F311881248C3680BB103F09E
:1007100087FA114A0F4800234FF47A7103F044FA24
:10072000002383F311880D4C236813B12368013B28
:100730002360636813B16368013B6360084B1B78F7
:1007400033B9636823B9022001F0ECF93223636006
:1007500010BD00BF50230020010700086C240020BA
:1007600064230020274B284A10B51C461968013124
:1007700046D004339342F9D16268244B9A423FD960
:10078000234B9B6803F1006303F580339A4237D211
:1007900003F0DAFD03F0ECFD002001F0F3F81D4B4F
:1007A0000220187001F0B4F91B4B1A6C00221A6475
:1007B000196E1A66196E596C5A64596E5A665A6ED9
:1007C0005A6942F080025A615A6922F080025A61E5
:1007D0005A691A6942F000521A611A6922F00052ED
:1007E0001A611B6972B64FF0E0232021C3F8084D4F
:1007F000D4E9003281F311889D4683F308881047BD
:1008000010BD00BF0000010820000108FFFF000824
:100810000023002064230020003802402DE9F04F1F
:1008200093B0AC4B00902022FF210AA89D6801F0F4
:10083000A9F9A94A1378A3B9A8480121C360117086
:10084000202383F31188C3680BB103F0E9F9A44AAC
:10085000A24800234FF47A7103F0A6F9002383F332
:100860001188009B9F4A03B113609F49009C00239D
:100870000B70536098469B461E469A46012001F035
:1008800047F924B1974B1B68002B00F01C82002015
:1008900001F030F80390039B002B01DA00F0CEFE4C
:1008A000039B002BEDDB012001F028F9039B213B8A
:1008B000162BE3D801A252F823F000BF1909000853
:1008C00041090008D50900087D0800087D080008D6
:1008D0007D080008690A00083B0C0008550B000859
:1008E000B70B0008DF0B0008050C00087D080008A6
:1008F000170C00087D080008890C0008B9090008D9
:100900007D080008CD0C000825090008B909000879
:100910007D080008B70B00080220FFF7DDFE002865
:1009200040F0FB81009B0221B8F1000F08BF1C467C
:1009300005A841F21233ADF8143000F0F9FF9DE73D
:100940004FF47A7000F0D6FF071EEBDB0220FFF7B2
:10095000C3FE0028E6D0013F052F00F2E081DFE86A
:1009600007F0030A0D10133605230593042105A88B
:1009700000F0DEFF17E057480421F9E75B48042147
:10098000F6E75B480421F3E74FF01C09484600F006
:10099000FBFF09F104090590042105A800F0C8FF38
:1009A000B9F12C0FF2D1012000FA07F747EA0B0B3F
:1009B0005FFA8BFB4FF0000A01F030F926B10BF023
:1009C0000B030B2B08BF0024FFF78EFE56E74948A8
:1009D0000421CDE7002EA5D00BF00B030B2BA1D1EA
:1009E0000220FFF779FE074600289BD001203E4EEB
:1009F00000F0C8FF0220307001F08AF84FF00008C4
:100A00005FFA88F9484600F0CDFF044690B14846A9
:100A100000F0D8FF08F101080028F1D1B8460446DB
:100A200041F21213022105A8ADF814303E4600F041
:100A30007FFF23E701230220337001F05FF8254692
:100A4000244B9B68AB4207D9284600F09DFF01303C
:100A500040F068810435F3E7234B00251D70214BDE
:100A6000B8465D603E46A7E7002E3FF45BAF0BF053
:100A70000B030B2B7FF456AF1B4B0220187001F0B9
:100A800047F8322000F036FFB0F10009FFF64AAF18
:100A900019F003077FF446AF0E4A926809EB05038D
:100AA00093423FF63FAFB9F5807F3FF73BAF124B24
:100AB0000193B94522DD4FF47A7000F01BFF0390DB
:100AC000039A002AFFF62EAF019B039A03F8012B2D
:100AD0000137EDE700230020682400205023002088
:100AE000010700086C240020642300200423002058
:100AF000082300200C23002068230020C820FFF7D3
:100B0000EBFD074600283FF40DAF1F2D11D8C5F1AE
:100B100020024A450AAB25F0030028BF4A46834914
:100B20000192184401F008F8019A8048FF2101F071
:100B300029F84FEAA9037D490193C9F387022846A2
:100B400001F028F8064600283FF46AAF019B05EB48
:100B5000830531E70220FFF7BFFD00283FF4E2AE36
:100B600000F05AFF00283FF4DDAE0027B946704B75
:100B70009B68BB4218D91F2F11D80A9B01330ED096
:100B800027F0030312AA134453F8203C0593484668
:100B9000042205A901F0C0F804378146E7E738468A
:100BA00000F0F2FE0590F2E7CDF81490042105A8BC
:100BB00000F0BEFE00E70023642104A8049300F0C7
:100BC000ADFE00287FF4AEAE0220FFF785FD0028C1
:100BD0003FF4A8AE049800F007FF0590E6E7002375
:100BE000642104A8049300F099FE00287FF49AAED3
:100BF0000220FFF771FD00283FF494AE049800F046
:100C000003FFEAE70220FFF767FD00283FF48AAE02
:100C100000F012FFE1E70220FFF75EFD00283FF43D
:100C200081AE05A9142000F00DFF042107460490B1
:100C300004A800F07DFE3946B9E7322000F05AFEE4
:100C4000071EFFF66FAEBB077FF46CAE384A9268A2
:100C500007EB0A0393423FF665AE0220FFF73CFD27
:100C600000283FF45FAE27F003075744BA453FF42E
:100C7000A3AE504600F088FE0421059005A800F0C0
:100C800057FE0AF1040AF1E74FF47A70FFF724FDEA
:100C900000283FF447AE00F0BFFE002844D00A9B76
:100CA00001330BD008220AA9002000F073FF0028AE
:100CB0003AD02022FF210AA800F064FFFFF714FDBC
:100CC0001C4802F02DFF13B0BDE8F08F002E3FF45A
:100CD00029AE0BF00B030B2B7FF424AE0023642111
:100CE00005A8059300F01AFE074600287FF41AAE07
:100CF0000220FFF7F1FC814600283FF413AEFFF716
:100D0000F3FC41F2883002F00BFF059800F0B8FFC9
:100D10004E4600F083FF3C46B0E506464CE64FF0F9
:100D2000000AFFE5B8467BE6374679E668230020EF
:100D300000230020A0860100094A136849F26900D7
:100D400099B21B0C00FB01331360064B186844F288
:100D5000506182B2000C01FB0200186080B2704743
:100D60001C2300201823002010B500211022044667
:100D700000F008FF034B03CB206061601868A0609F
:100D800010BD00BF107AFF1F2DE9F043204DBBB00E
:100D900000F0BEFFAB68C31AF92B32D906AFA860CA
:100DA0002B4628220021384601F04AFC05F10E00AE
:100DB00000F0E0FE002604465FFA80F905F10E0817
:100DC000F3B2F100994501F1280107D908EB0603B8
:100DD0000822384601F034FC0136F1E708230122ED
:100DE000CDE9023205340B4B0193A4B230230093BA
:100DF000CDE9047404A3D3E90023297B064801F05C
:100E000037FA3BB0BDE8F08378F6339F93CACD8DB7
:100E1000B0340020BD3400208C34002070B50D4665
:100E200014461E4601F0BAF950B9022E10D1012C19
:100E30000ED112A3D3E90023C5E90023012007E066
:100E4000282C10D005D8012C09D0052C0FD000205B
:100E500070BD302CFBD10BA3D3E90023ECE70BA32F
:100E6000D3E90023E8E70BA3D3E90023E4E70BA3CE
:100E7000D3E90023E0E700BFAFF30080401DA120CD
:100E800026812A0B78F6339F93CACD8D9E6AC421A2
:100E9000818A46EE26417272DF25D7B7F017304AB5
:100EA00039059E5613B504462346084620220021E4
:100EB000019001F0C5FB22790198032A234628BF3F
:100EC000032203F8042F2021022201F0B9FB6279EA
:100ED0000198072A234628BF072203F8052F22215D
:100EE000032201F0ADFBA2790198072A234628BF0F
:100EF000072203F8062F2521032201F0A1FB019808
:100F000004F108031022282101F09AFB382002B0D6
:100F100010BD00002DE9F04FADF5037D23AD10AEFF
:100F200040F2751280460F4624A80021296000F087
:100F300029FE48220021304600F024FE00F0E8FEA1
:100F4000564B4FF47A72B0FBF2F0186093E807004A
:100F5000012386E807000DF162003382FFF704FFEA
:100F60004FF20363338407AB18464D4904F0C4FBCA
:100F70004FF0200930642946304686F83C90FFF750
:100F800091FF14AB044601460822284601F058FBA5
:100F90000822A1180DF15103284601F051FB0DF173
:100FA0005203082204F11001284601F049FB4A4689
:100FB00015AB04F11801284601F042FB16AB4022A4
:100FC00004F13801284601F03BFB18AB082204F17C
:100FD0007801284601F034FB0DF16103082204F189
:100FE0008001284601F02CFB04F1880A0DF162090A
:100FF00004F5847B4B465146082228460AF1080A2C
:1010000001F01EFBD34509F10109F3D11DAB082204
:101010005946284601F014FB04F588744FF0000986
:1010200096F834304B450AD9B36B21464B4408221D
:10103000284601F005FB083409F10109F0E74FF0FB
:10104000000996F83C304B4504EBC90108D9336CD4
:1010500008224B44284601F0F3FA09F10109F0E7B0
:10106000CB1DC3F3CF03CDE9045300230393BB7E11
:10107000029307F11903019301230093F97E05A35D
:10108000D3E90023404601F0F3F80DF5037DBDE8F8
:10109000F08F00BF9E6AC421818A46EE742400202E
:1010A00008570008014B1870704700BF80240020CB
:1010B000F0B5334B1C7B85B034B1324B0E221A8114
:1010C0000024204605B0F0BD2F4A1068516802ABDD
:1010D00003C308232D492E480DEB030204F0EAFA5E
:1010E000054630B9274B2B480A221A8100F0CAFD69
:1010F000E6E70169B1F5702F06D9224B26480B228D
:101100001A8100F0BFFDDCE7438B40F2F6329342D8
:1011100007D01C490C2008811946204800F0B2FD78
:10112000CFE71F4A024402F11003994204D2154B43
:101130001C4810221A81E4E710398E1A20461449FF
:1011400000F0EAFD3246074605F11801204600F09E
:10115000E3FDAB689F4202D1EB6898420AD0094B8D
:101160000D221A810090D5E902123B460E4800F08C
:1011700089FDA5E70D4800F085FD0124A1E700BF2A
:10118000B034002074240020BD570008DCFF0E009E
:10119000000001082C570008385700084A5700087B
:1011A0000800FFF76857000885570008AE57000889
:1011B0002DE9F04FADB006AF80460C4600F0EEFFD3
:1011C000054600285AD1237E022B1BD1E38A012B2E
:1011D00018D100F09DFD0646FFF7AEFD03464FF423
:1011E000C870DFF8D092B3FBF0F206F5167602FB7A
:1011F000103316FA83F3C9F80030E37E33B9A84BF5
:1012000000221A709C37BD46BDE8F08FA38AEEB26B
:10121000013BB34205F101050BD93B1D1E44E9001A
:1012200000960023082201F0F801204601F0CCF8D6
:10123000ECE707F11400FFF797FD324607F11401C0
:10124000381D04F027FA0028D9D10F2E08D8944B66
:101250001E70D9F80030A3F51673C9F80030D1E735
:10126000FB1CF8700146009307220346204601F05C
:10127000ABF8F978404600F089FFC3E7E38A282BF2
:1012800026D010D8012B1ED0052BBBD1BFF34F8F1A
:101290008449854BCA6802F4E0621343CB60BFF314
:1012A0004F8F00BFFDE7302BACD1637E7F4D013304
:1012B0006A7BDBB29342E94603D1E27E2B7B9A4202
:1012C00065D0CD469EE721464046FFF723FE99E7CD
:1012D000A38A013B9BB2C92B94D8744D2E7B26BBAD
:1012E00005F10C030093082233463146204601F0F5
:1012F0006BF8731CF2B2D9001E46A38A013B9A42D6
:1013000005DA0E322A44009200230822EEE7002379
:101310000022C5E900230023AB6085F8D730C5F86B
:10132000D8302B7B0BB9E37E2B73002507F1140912
:101330003B1D082229464846C7E90155FD6001F0DA
:101340007FF93B7A05F1010AAB424FEACA0608D998
:10135000FB6808222B443146484601F071F9554696
:10136000EFE7C6F3CF06E17ECDE9049600230393B1
:10137000A37E0293193428230093019446A3D3E952
:101380000023404600F074FFFFF7FEFC3AE74FF001
:10139000000807F11403A7F81480102200934146B7
:1013A0000123204601F010F8A68A023EB6B2F31CD3
:1013B0009B109B000733DB08A9EBC3039D460DF18F
:1013C000180A1FFA88F34FEAC801B34201F110016D
:1013D0000AD20AEB0803009308220023204600F0FB
:1013E000F3FF08F10108ECE795F8D70000F0DAFA0E
:1013F000D5F8D83004461BB995F8D70000F0E2FACA
:10140000D5F8D83033449C4204D295F8D700013047
:1014100000F0D8FA4FEA960B4FF000081FFA88F157
:101420008B45D5E9003209D90AEB880103EB880026
:10143000012200F0AFFB08F10108EFE7F31842F1D9
:101440000002C5E90032D5F8D83095F8D70006EB90
:101450000308C5F8D88000F0A5FA804509D395F8AF
:10146000D730D5F8D8000133001B85F8D730C5F840
:10147000D800FF2E08D800232B7300F0CDFAFFF719
:1014800017FE08B1FFF76EF92B68094A9B0A013372
:1014900013810023AB6014E726417272DF25D7B7B2
:1014A0008534002000ED00E00400FA05B03400208F
:1014B000742400208834002008B54FF000530B4AF4
:1014C000196891420AD10A4A597D117009481B7D59
:1014D00003730949C9220E3000F02EFBBDE8084015
:1014E000E02200214FF0005000F04CBB9AAD44C503
:1014F00080240020B0340020160000202DE9FF4198
:10150000434C02236371002302932A250A23581EA9
:10151000B5FBF3F67343D3F12A02C1B23ED00228E1
:101520000346F4D19DF80B303A493B485A1E9DF8CA
:101530000A30013B1B0443EA0253BDF80820013A7C
:1015400013434B6001F028FD00230193334B3449D2
:1015500000933448344B4FF4805200F0F1FD334B8C
:10156000197811B12F4800F011FE00F0D1FB0546AB
:10157000FFF7E2FB4FF4C873B0FBF3F202FB130377
:1015800005F5167010FA83F0294B186002F012FF6F
:1015900008B10F23238104B0BDE8F081C1EBC1077E
:1015A000FB1C4FEAE30EC3F3C703A1EB030C0EF1E0
:1015B00001084FF47A705FFA8CF50EFB000058FAC0
:1015C0008CFCB0FBFCF0B0F5617F07D97B1EC3F348
:1015D000C703C91ACDB2591E0F2916D86A1E072A89
:1015E0008CBF00220122591901FB06601149B1FB91
:1015F000F0F11148814295D1002A93D0ADF80860EE
:101600008DF80A308DF80B508CE71346EBE700BFDE
:101610007424002010230020C83500201D0E00086F
:10162000842400208C340020B11100088024002084
:101630008834002080DE800240420F002DE9F04F08
:1016400091A7D7E900670FF24829D9E90089874DAA
:1016500093B0DFF844B2864C284600F06DFE0DF1E1
:10166000300A079070B310220021504600F08AFA29
:10167000079B197B4FF0000261F303028DF83020C5
:10168000586899680EAA03C21B680D9A63F31C027E
:101690009DF830300D9243F020038DF83030002358
:1016A00052461946584601F087FC079028B928464B
:1016B00000F046FE079B2370CEE72378072B3CD82B
:1016C0000133237018220021504600F05BFADFF846
:1016D000C8B1684C002319465246584601F094FCA4
:1016E000014670BB102208A800F04CFA636983F42D
:1016F0008043636100F00EFB0B4612A9024611E91C
:1017000003000DF1240C8CE803009DF83410C1F3A4
:10171000030089064CBF0E99BDF838C08DF82C0027
:1017200046BFC1F31C0C4CF00041CCF30A010891F8
:10173000284608A900F0CCFFCCE7284600F000FEC0
:10174000C0E7284600F02AFD0446002848D1DFF80B
:101750004CB100F0DDFADBF80030984240D300F0E5
:10176000D7FA0790FFF7E8FA079A8DF8204003466A
:101770004FF4C87002F51672B3FBF0F101FB1033A1
:1017800012FA83F3CBF80030DFF814B19BF80010A5
:1017900011B901238DF8203050460791FFF7E4FA84
:1017A0000799C1F11004E4B2062C28BF0624224692
:1017B00051440DF1210000F0BFF908AB0393182349
:1017C000029301342C4B0193E4B20123009304945F
:1017D0003B463246284600F0E3FC00238BF80030FD
:1017E00000F096FA254A264C1368C31AB3F57A7F9F
:1017F00031D3106000F08EFA02460B46284600F006
:10180000A9FD284600F0CAFC28B3237BDFF894B07A
:10181000002B14BF032302238BF8053000F078FA65
:101820004FF47A735146B0FBF3F0CBF80000584602
:10183000FFF738FB182307300293124B0193C0F3D4
:10184000CF0040F25513CDE903A0009342464B462A
:10185000284600F0A5FC237B2BB1FFF795FA237BEC
:10186000002B7FF4F6AE13B0BDE8F08F8C3400206F
:10187000953500200000024084340020903500207F
:10188000B034002094350020401DA12026812A0B71
:10189000F1C6A7C1D068080FC835002088340020E1
:1018A000853400207424002070B50F4B1B78013361
:1018B000DBB2012B0C4611D80C4D29684FF47A731A
:1018C0000E6AA2FB0332014622462846B0478442F4
:1018D00004D1074B00221A70012070BD4FF4FA703A
:1018E00002F01EF90020F8E720230020B037002086
:1018F000C435002007B50023024601210DF1070081
:101900008DF80730FFF7D0FF20B19DF8070003B036
:101910005DF804FB4FF0FF30F9E700000A4608B518
:101920000421FFF7C1FF80F00100C0B2404208BDB2
:1019300030B4054C2368DD69044B0A46AC460146C9
:10194000204630BC604700BFB0370020A0860100B1
:1019500070B502F095FB094E094D308000242868CF
:101960003388834208D902F085FB2B680444013395
:10197000B4F5803F2B60F2D370BD00BFC6350020A8
:101980009835002002F02ABC00F1006000F580309C
:101990000068704700F10060920000F5803002F0AE
:1019A000B5BB0000054B1A68054B1B889B1A834288
:1019B00002D9104402F05EBB002070479835002029
:1019C000C635002038B5074D04462868204402F08B
:1019D00059FB28B928682044BDE8384002F06ABBAA
:1019E00038BD00BF9835002010F003030AD1B0F5D0
:1019F000047F05D200F10050A0F51040D0F8003867
:101A0000184670470023FBE700F10050A0F5104096
:101A1000D0F8100A70470000064991F8243033B11D
:101A20000023086A81F824300822FFF7B3BF0120A1
:101A3000704700BF9C350020014B1868704700BFFD
:101A4000002004E070B52A4B1B68C3F30B02044668
:101A50001B0C62B140F21340824230D040F2194078
:101A600082422ED040F2214082422CD10322214DCD
:101A70000C2000FB0252556842F20102934224D02E
:101A8000B3F5805F23D041F20102934221D041F2AD
:101A9000030293421FD041F20702934214BF3F2337
:101AA0003123013C0C44013D0A46A24215D215F9EE
:101AB000016F501C9EB100F8016C0246F5E701224F
:101AC000D5E70222D3E70C4DD6E73323E9E74123DC
:101AD000E7E75A23E5E75923E3E7104605E02C251D
:101AE0008442157001D9901C5370401A70BD00BF1C
:101AF000002004E0F4570008C8570008022802BF7D
:101B0000024B4FF080429A61704700BF00000240D4
:101B1000022802BF024B4FF480429A61704700BF17
:101B200000000240022801BF024A536983F4804347
:101B3000536170470000024010B50023934203D068
:101B4000CC5CC4540133F9E710BD000010B5013876
:101B500010F9013F3BB191F900409C4203D11AB109
:101B60000131013AF4E71AB191F90020981A10BD39
:101B70001046FCE703460246D01A12F9011B002961
:101B8000FAD1704702440346934202D003F8011B86
:101B9000FAE770472DE9F8431F4D144695F82420C5
:101BA0000746884652BBDFF870909CB395F8243006
:101BB0002BB92022FF2148462F62FFF7E3FF95F85B
:101BC0002400C0F10802A24228BF2246D6B24146F4
:101BD000920005EB8000FFF7AFFF95F82430A41BBF
:101BE0001E44F6B2082E17449044E4B285F82460EF
:101BF000DBD1FFF711FF0028D7D108E02B6A03EBF8
:101C000082038342CFD0FFF707FF0028CBD100200B
:101C1000BDE8F8830120FBE79C350020024B1A78D1
:101C2000024B1A70704700BFC435002020230020EB
:101C300010B50F4C0F4801F089FA21460D4801F00C
:101C4000B1FA24680C48626DD2F8043843F00203FC
:101C5000C2F8043801F064FF0849204601F0A8FBEF
:101C6000626DD2F8043823F00203C2F8043810BDC4
:101C7000E8580008B037002040420F00F058000834
:101C8000704700000FB4002004B0704700B59BB04F
:101C9000EFF3098168226846FFF74EFFEFF30583F3
:101CA000044B9A6BDA6A9A6A9A6A9A6A9A6A9A6A88
:101CB0009B6AFEE700ED00E000B59BB0EFF3098101
:101CC00068226846FFF738FFEFF30583044B9A6BF1
:101CD0009A6A9A6A9A6A9A6A9A6A9B6AFEE700BF47
:101CE00000ED00E000B59BB0EFF309816822684683
:101CF000FFF722FFEFF30583034B5A6B9A6A9A6A48
:101D00009A6A9A6A9B6AFEE700ED00E0FEE700002F
:101D100002F09EBA02F076BA30B5094D0A449142FB
:101D20000DD011F8013B5840082340F30004013B5B
:101D30002C4013F0FF0384EA5000F6D1EFE730BDEA
:101D40002083B8ED2DE9F041C56915B9C161BDE841
:101D5000F0814B6823F06047C3F38A464FEAD37E95
:101D6000C3F3807816EA230638BF3E46AC462B46BE
:101D70005A68BEEBD27F22F060440AD0002A18DAFB
:101D8000A40CB44217D19D420FD10D60DEE713467B
:101D9000EEE7A74207D102F08044C2F380724245C9
:101DA0000BD054B1EFE708D2EDE7CCF800100B6090
:101DB000CDE7B44201D0B442E5D81A689C46002A67
:101DC000E5D11960C3E700002DE9F047089D01F057
:101DD00007044FEAD508224405F0070500EBD100BF
:101DE0004FF47F49944201D1BDE8F08704F0070722
:101DF00005F0070A57453E4638BF5646C6F1080665
:101E0000111B8E4228BF0E46E10808EBD50E415C3F
:101E100013F80EC0B94029FA06F721FA0AF1FFB209
:101E20008CEA010147FA0AF739408CEA010C03F801
:101E30000EC034443544D5E780EA0120082341F23E
:101E4000210201B24000002980B203F1FF33B8BF84
:101E5000504013F0FF03F4D17047000038B50C4632
:101E60008D18A54200D138BD14F8011BFFF7E4FF1F
:101E7000F7E7000002684AB113680360C38801896C
:101E800001339BB29942C38038BF0381104670472B
:101E900070B588B0202204460D4668460021FFF741
:101EA00071FE20460495FFF7E5FF024658B16B46E8
:101EB000054608AE1C4603CCB44228606960234640
:101EC00005F10805F6D1104608B070BD10B54B6895
:101ED00023B9CA8A63F30902CA8210BDC4681A68AA
:101EE0001C60C360438A013B43824A60EFE7000005
:101EF0002DE9F84F1D46CB8A0F46C3F30901062989
:101F0000814692460B4630D00020AAB207F1190450
:101F10009EB2052E1FFA80F80FD8904503F10103F9
:101F200006D3FB8A0A4462F30903FB8201201AE00C
:101F30001AF80060E6540130EAE79045F1D2A1F1C9
:101F4000060B1C237C68BBFBF3F203FB12BB1FFADE
:101F50008BF6002C45D14846FFF78CFF044638B974
:101F600078606FF00200BDE8F88F4FF00008E6E7F8
:101F7000002606607860ADB24FF0000B454510D9E1
:101F80000AEB0803221D13F8011B9155B1B208F1A9
:101F900001081B291FFA88F82BD0454506F10106D8
:101FA000F1D8FB8AC3F30902154465F30903BCE7C2
:101FB000013292B21C462368002BF9D1AB1F0B44AF
:101FC0001C21B3FBF1F301339BB29A42D3D2BBF194
:101FD000000FD0D14846FFF74DFF20B9C4F800B03C
:101FE000BFE70122E7E7C0F800B05E462060044684
:101FF000C1E74545D5D94846FFF73CFF08B9206001
:10200000AFE7C0F800B0002620600446B6E7000045
:102010002DE9F04F2DED028B83B0CDE90013BDF813
:102020003C4080469246002A00F087802CB10E9BEF
:10203000002B00F08280072C2BD808F10C00FFF752
:1020400019FF054638B96FF00205284603B0BDEC0C
:10205000028BBDE8F08F14220021FFF793FD22468A
:102060000E9905F10800FFF767FD631C2B749AF8C1
:1020700000302C4403F01F0363F03F032372009BE6
:1020800043F00041696040462946FFF75BFE0125A9
:10209000DBE700F10C034FF0000908EE103A4FF0B7
:1020A000800B4E464D4618EE100AFFF7E3FE07463A
:1020B0000028C8D014220021FFF764FD002E3AD179
:1020C000019B3B8102220E9B02F1080103EB060CEF
:1020D00057FA81F11046B44202F10102D2B201D89E
:1020E000024607E01CF8010B01F8010B0136062A35
:1020F000B6B2EFD99AF8001001F01F01B44208BF40
:102100004FF0400BB81841EA49114BEA0103037242
:10211000009B013243F000437B603A7439464046ED
:10212000FFF710FE0135B4422DB289F001094FF0DE
:10213000000BB8D189E70022C5E76FF0010584E7FD
:10214000F8B515460E462422002104461F46FFF727
:1021500019FD069B6360B5F5001F079BA76034BFA0
:102160006A094FF6FF72236204F10C0097B2002354
:102170009A4205D80023036027826382A382F8BDB8
:102180000660013330462036F2E7000003781BB9C1
:102190004BB2002BC8BF0170704700000078704739
:1021A0002DE9F74FDDF83C90BDF830500D9E9DF8BD
:1021B0003840BDF84070804692469B46B9F1000F0A
:1021C00001D1002F51D11F2C4FD898F80000B0B981
:1021D000072F47D835F0030347D13A4649464FF613
:1021E000FF70FFF73BFE20F001002D02400445EA9E
:1021F0000464400C44EA40244FF6FF7321E040EAB7
:102200000520072F40EA0464F6D900254FF6FF7336
:10221000C5F12000A5F120022AFA05F10BFA00F021
:1022200001432BFA02F211431846C9B2FFF704FE2C
:102230000835402D0346EBD13A464946FFF70EFEDE
:102240000346CDE90097324621464046FFF7E0FEBF
:1022500033780133DBB21F2B88BF0023337003B008
:10226000BDE8F08F6FF00300F9E76FF00100F6E7CB
:102270002DE9F04F85B09246DDF848800F9D9DF81E
:1022800040209DF84490BDF84C7006469B46B8F13E
:10229000000F01D1002F48D11F2A46D83378002BD8
:1022A00046D00C0244EA02649DF8381044EAC9346E
:1022B00044EA01441C43072F44F0800432D9002330
:1022C0004FF6FF72C3F1200CA3F120002AFA03F1AC
:1022D0000BFA0CFC41EA0C012BFA00F00143C9B2E5
:1022E00010460393FFF7A8FD039B0833402B0246DB
:1022F000E8D13A464146FFF7B1FD0346CDE90087F4
:102300002A4621463046FFF783FEB9F1010F06D178
:102310002B780133DBB21F2B88BF00232B7005B055
:10232000BDE8F08F4FF6FF73E8E76FF00100F6E7C6
:102330006FF00300F3E70000C06900B1043070479C
:10234000C3691A68C261C2681A60C360438A013BEC
:10235000438270472DE9F041D0F81880194E144699
:102360001D464146002709B9BDE8F081D1E90223A5
:10237000A21A65EB0303964277EB03031ED283692F
:102380008B420DD1FFF7A2FD83691B688361C3688F
:102390000B60438AC1608169013B43828846E2E762
:1023A000FFF794FD0B68C8F80030C3680B60438AE0
:1023B000C160013B4382D8F80010D4E78846096821
:1023C000D1E700BF80841E002DE9F04F8BB00D4691
:1023D000DDF8509014469B468046002800F0198195
:1023E000B9F1000F00F01581531E3F2B00F211814F
:1023F000012A03D1BBF1000F40F00B810023CDE98E
:102400000833B8F81430B5EBC30F4FEAC30703D352
:1024100000200BB0BDE8F08F2B199F42D8F80C308C
:102420003ABF7F1BFFB227461BB9D8F81030002BEC
:102430007AD02F2D4ED8C5F13006B7424FF00003A9
:102440002CBFF6B23E4600932946D8F8080008ABE8
:102450003246FFF7B9FCA7EB060A35445FFA8AFA61
:10246000B8F8143003F10053063BDB000493D8F8AE
:102470000C3003933021039B13B1BAF1000F2CD120
:10248000D8F8100040B1BAF1000F05D0009608ABA3
:102490005246691AFFF798FC38B2002FB8D0660789
:1024A0000AD00AAB03EBD401624211F8083C02F0F7
:1024B0000702134101F8083C082C3CD9102C40F2CB
:1024C000B580202C40F2B780BBF1000F00F09C805B
:1024D000082334E0BA460026C2E7049BE02B28BF5D
:1024E000E02306930B44AB42059314D95A1B03987F
:1024F0000096924534BF5246D2B2691A08AB0430F6
:102500000792FFF761FC079A1644AAEB020A1544EA
:10251000F6B25FFA8AFA049B069A05999B1A04930D
:10252000039B1B680393A6E70093D8F8080008AB49
:102530003A462946AEE7BBF1000F13D00123B4EBB6
:10254000C30F6CD0082C12D89DF82030621E23FADD
:1025500002F2D50706D54FF0FF3202FA04F4234306
:102560008DF820309DF8203089F8003051E7102C8C
:1025700012D8BDF82030621E23FA02F2D10706D528
:102580004FF0FF3202FA04F42343ADF82030BDF8D7
:102590002030A9F800303CE7202C0FD80899631EA2
:1025A00021FA03F3DA0705D54FF0FF3202FA04F4FB
:1025B0000C430894089BC9F800302AE7402C2BD024
:1025C000DDE90865611EC4F12102A4F1210326FAA8
:1025D00001F105FA02F225FA03F311431943CB077F
:1025E00012D50122A4F12003C4F1200102FA03F361
:1025F00022FA01F1A240524243EA010363EB430392
:1026000032432B43CDE90823DDE90823C9E9002340
:10261000FFE66FF00100FCE66FF00800F9E6082C19
:10262000A0D9102CB3D9202CEED8C3E7BBF1000FF2
:10263000ADD0022383E7BBF1000FBBD004237EE7BC
:1026400030B5012A144638BF0124402C85B028BF7C
:1026500040240025012ACDE9025518D81B788DF8B1
:10266000083063070AD004AB03EBD405624215F8C7
:10267000083C02F00702934005F8083C009103462D
:102680002246002102A8FFF79FFB05B030BD082AB3
:10269000E4D9102A03D81B88ADF80830E1E7202AD6
:1026A0008DBFD3E900231B680293CDE90223D8E74D
:1026B00010B5CB681BB98B600B618B8210BDC468F1
:1026C0001A681C60C360438A013B4382CA60F0E71A
:1026D0002DE9F04FD1F8008093B018F0800FCDE9CC
:1026E0000323C8F3C01219BFC8F3C03BC8F30626C2
:1026F0004FF0020B1646B8F1000F04460D4680F26B
:10270000C58118F0C043059340F0C0810B7B002BBE
:1027100000F0BC81BBF1020F03D00178B14240F060
:10272000B88108F07F0106916AB3C8F3074A2B44C9
:10273000069A93F80390760646EA0B4646EA8246E6
:102740005FEAD91346EA0A06079300F09080002258
:102750000023CDE90A23069B009367685B46524637
:102760000AA92046B84700287ED0A7699FB93146FC
:1027700004F10C00FFF78CFB0746E0B96FF0020094
:1027800013B0BDE8F08FC8F30F2A18F07F0F08BF11
:102790000AF0030ACBE73B699E420DD03F68002F49
:1027A000F9D1314604F10C00FFF772FB074600280F
:1027B000E4D0A3693B60A761DDE90A2300264FF658
:1027C000FF70C6F1200E22FA06F103FA0EFEA6F102
:1027D000200C23FA0CFC41EA0E0141EA0C01C9B2BB
:1027E000083609920893FFF727FB402EDDE90832EF
:1027F000E7D1B882FB7D09F01F06C3F38403F31A07
:10280000D7E9022198B2002BBCBF00F120031BB214
:1028100052EA0100C8F304680FD00398821A0498A2
:1028200060EB0101A14890424FF000028A4104D3BD
:10283000079A002A55D0012B23DDFA7D4FEA890340
:1028400002F0030203F07C031343FB753946204674
:10285000FFF73CFB079BA3B9FB7DC3F38402013266
:1028600062F38603FB7504E06FF00B0088E7A7694D
:1028700017B96FF00C0083E73B699E42BAD03F68FE
:10288000F6E719F0400F2CD0039BBB60049BFB6064
:10289000142200210DA8FFF775F9039B0A93049BEE
:1028A0000B932B1D0C932B7BADF83EA0013BDBB2B1
:1028B000ADF83C30069B8DF843308DF840B0A368EE
:1028C0008DF841608DF842800AA920469847FB7D2B
:1028D000C3F38403013303F01F039B02FB82002038
:1028E0004EE7FB7DC9F34012B2EBD31F40F0D4801A
:1028F000C3F38403B34240F0D28007992B7B4FEAA5
:102900009912002934D0D20741D4032B40F2CA8057
:10291000039BBB60049BFB602B7BAE1D033BDBB2C8
:102920003246394604F10C00FFF7E2FA00280DDACE
:1029300020463946FFF7CAFAFB7DC3F3840301330F
:1029400003F01F039B02FB82032019E7AB883B8344
:102950002A7B033AB88AD2B23146FFF77FFAFB7D71
:10296000B882DA43C2F3C01262F3C713FB75B6E74D
:102970006AB92E1D013BDBB23246394604F10C0028
:10298000FFF7B6FA0028D3DB2A7B013AE2E7F98A9F
:10299000C1F30901013B0529DAB253D8281D0023F0
:1029A00007F11A0C9A4208D910F801EB0CF801E073
:1029B000013101330629DBB2F4D103990A9104995C
:1029C0000B91934207F11A010C9138BF04337968D7
:1029D0000D9134BF55FA83F300230E93FB8AADF8B3
:1029E0003EA0C3F309031A44069B8DF8433000232D
:1029F000ADF83C208DF840B08DF841608DF84280F4
:102A00007B602A7BB88A013A291DFFF727FA3B8BA6
:102A1000B882834203D1A3680AA92046984720467A
:102A20000AA9FFF745FEFB7DB88AC3F3840301338F
:102A300003F01F039B02FB823B8B984214BF1120C3
:102A400000209DE67B68002BB7D0062001E01C30FB
:102A50006346D3F800C0BCF1000FF8D1091A081D75
:102A600005F1040C00EB030905989DF8143001EB07
:102A7000000EBEF11B0FA0D89A429ED91CF8013B54
:102A800009F8013B059B01330593EDE76FF0090061
:102A900076E66FF00A0073E66FF00D0070E66FF0F7
:102AA0000E006DE66FF00F006AE600BF80841E0026
:102AB000404BF0B51C6C404E44F000741C641D6E1D
:102AC00045F000751D661B6E3C4B9B6AD3F80052A7
:102AD000354045F00105C3F80052D3F800423440B8
:102AE00044EA002040F00100C3F80002002952D05F
:102AF0000020C3F81C020546C3F80402C3F80C0208
:102B0000C3F8140203EBC00401301C28C4F840527F
:102B1000C4F84452F6D100254FF0010C9678148881
:102B2000F70748BFD3F804720CFA04F044BF074318
:102B3000C3F80472B70742BFD3F80C720743C3F857
:102B40000C72760742BFD3F814620643C3F81462CE
:102B500003EBC4045668C4F840629668C4F8446243
:102B6000D3F81C4201352043A942C3F81C0202F1EC
:102B70000C02D3D1D3F8002222F00102C3F80022C4
:102B80000C4B1A6C22F000721A641A6E22F000725A
:102B90001A661B6EF0BD0122C3F84012C3F844123E
:102BA000C3F80412C3F81412C3F80C22C3F81C2291
:102BB000E0E700BF003802400000FFFFC8350020FA
:102BC000184A916A08B58B688B6013F0010104D034
:102BD00013F00C0F18BF4FF48031D80506D513F44D
:102BE000406F14BF41F4003141F00201D80306D513
:102BF00013F4402F14BF41F4802141F00401D36944
:102C00000BB108489847202383F311880648002118
:102C100000F0AEFF002383F31188BDE8084001F007
:102C200003BC00BFC8350020D035002038B5124C99
:102C3000A36ADD68AA0712D05A6922F002025A611B
:102C4000A36913B1012120469847202383F31188FB
:102C50000A48002100F08CFF002383F31188EB0663
:102C600006D5A36A1021D960236A0BB102489847A0
:102C7000BDE8384001F0D8BBC8350020D835002069
:102C800038B5124CA36A1D69AA0712D05A6922F0FE
:102C900010025A61A36913B10221204698472023EC
:102CA00083F311880A48002100F062FF002383F3B8
:102CB0001188EB0606D5A36A10211961236A0BB1AE
:102CC00002489847BDE8384001F0AEBBC835002047
:102CD000D835002038B50F4CA36A5D685D602A07BF
:102CE0000AD5042222701A6822F002021A60636A6E
:102CF00013B10021204698476B0706D5A36A99694E
:102D0000236A13B1034809049847BDE8384001F02D
:102D10008BBB00BFC835002010B50E4C204600F01C
:102D200029F90D4BA3620B21132000F00BF90B21A5
:102D3000142000F007F90B21152000F003F90B21F6
:102D4000162000F0FFF80022BDE8104011460E20CA
:102D5000FFF7AEBEC835002000640040114B98421A
:102D600010B5044609D1104B1A6C42F000721A6477
:102D70001A6E42F000721A661B6EA36A01221A6074
:102D8000A36A5A68D20707D5626851681268D96188
:102D90001A60064A5A6110BD0121082000F0D4FDD6
:102DA000EEE700BFC8350020003802405B87010015
:102DB00003291AD8DFE801F0020A0F14836A9B681E
:102DC00013F0E05F14BF012000207047836A986809
:102DD000C0F380607047836A9868C0F3C060704732
:102DE000836A9868C0F30070704700207047000045
:102DF00010B5032925D8DFE801F00225292D836AC3
:102E00009968C1F30161183103EB0113107884064E
:102E10004CBF54689488C0F300114FEA410148BF89
:102E200041EAC40100F00F004CBF41F0040141EA47
:102E30004451586041F001019068D2689860DA60AE
:102E4000196010BD836A03F5C073DFE7836A03F579
:102E5000C873DBE7836A03F5D073D7E701290AD08B
:102E600002290FD081B9836ADA68920701D1186903
:102E700003E001207047836AD86810F0030018BF90
:102E800001207047836AF2E70020704710B539B916
:102E9000836AD96889071BD11B699C0704D110BDBF
:102EA000012915D00229FAD1816AD1F8C031D1F8AF
:102EB000C441D1F8C8011061D1F8CC015061202083
:102EC00008610869800717D1486940F0100012E0D6
:102ED000816AD1F8B031D1F8B441D1F8B8011061AC
:102EE000D1F8BC0150612020C860C868800703D1B8
:102EF000486940F002004861C3F34000C3F3800119
:102F0000000140EA4111107920F0300001431171B5
:102F100089064BBF91681189DB085B0D4CBF63F3D9
:102F20001C0163F30A01137948BF916064F3030342
:102F300013714FEA14234FEA144458BF11811370E0
:102F40005480ACE700F1604303F561430901C9B265
:102F500083F80013012200F01F039A4043099B00ED
:102F600003F1604303F56143C3F880211A607047A1
:102F7000FFF7D2BE012300F10802C0E9022203706C
:102F800000F110020023C0E90422C0E90633C0E9C1
:102F9000083343607047000010B52023044683F3D4
:102FA0001188022303704160FFF7D8FE04232370C9
:102FB000002383F3118810BD2DE9F0411F4604461C
:102FC0000D461646202383F3118800F10808237864
:102FD000052B0DD029462046FFF7EAFE40B12046DA
:102FE00032462946FFF704FF002080F3118808E0ED
:102FF0003946404600F0A0FD0028E8D0002383F3C6
:103000001188BDE8F08100002DE9F0411F4604461B
:103010000D461646202383F3118800F1100823780B
:10302000052B0DD029462046FFF718FF40B120465A
:1030300032462946FFF72AFF002080F3118808E076
:103040003946404600F078FD0028E8D0002383F39D
:103050001188BDE8F08100000268436811430160F7
:1030600003B118477047000013B5446BD4F894348B
:103070001A681178042915D1217C022912D11979F5
:10308000128901238B4013420CD101A904F14C0099
:1030900001F088FFD4F89444019B2179024620680E
:1030A00000F0CEF902B010BD143001F00BBF0000EB
:1030B0004FF0FF33143001F005BF00004C3001F039
:1030C000DDBF00004FF0FF334C3001F0D7BF0000F0
:1030D000143001F0D9BE00004FF0FF31143001F080
:1030E000D3BE00004C3001F0A9BF00004FF0FF320A
:1030F0004C3001F0A3BF00000020704710B5D0F89D
:1031000094341A6811780429044617D1017C0229E5
:1031100014D15979528901238B4013420ED11430B6
:1031200001F06CFE024648B1D4F894444FF4807329
:1031300061792068BDE8104000F070B910BD000052
:10314000406BFFF7DBBF0000704700007FB5124BFC
:10315000036000234360C0E90233012502260F4BC0
:10316000057404460290019300F1840229460096FA
:103170004FF48073143001F01DFE094B0294CDE929
:10318000006304F523724FF48073294604F14C0068
:1031900001F0E4FE04B070BD24580008413100087D
:1031A000693000080B68202282F311880A7903EB4A
:1031B000820290614A79093243F822008A7912B179
:1031C00003EB8203986102230374C0F89414002374
:1031D00083F311887047000038B5037F044613B1AC
:1031E00090F85430ABB9201D01250221FFF734FFC0
:1031F00004F1140025776FF0010100F0B9FC84F8A8
:10320000545004F14C006FF00101BDE8384000F06B
:10321000AFBC38BD10B5012104460430FFF71CFFD8
:103220000023237784F8543010BD000038B50446DD
:103230000025143001F0D6FD04F14C00257701F093
:10324000A5FE201D84F854500121FFF705FF2046FC
:10325000BDE83840FFF752BF90F8443003F06003F8
:10326000202B07D190F84520212A4FF0000303D8E6
:103270001F2A06D800207047222AFBD1C0E90E334E
:1032800003E0034A82630722C2630364012070479C
:103290002123002037B5D0F894341A681178042916
:1032A00004461AD1017C022917D119791289012308
:1032B0008B40134211D100F14C05284601F026FF46
:1032C00058B101A9284601F06DFED4F89444019B41
:1032D00021790246206800F0B3F803B030BD000049
:1032E000F0B500EB810385B09E6904460D46FEB142
:1032F000202383F3118804EB8507301D0821FFF795
:10330000ABFEFB685B691B6806F14C001BB10190CA
:1033100001F056FE019803A901F044FE024648B1AF
:10332000039B2946204600F08BF8002383F3118885
:1033300005B0F0BDFB685A691268002AF5D01B8AF7
:10334000013B1340F1D104F14402EAE7093138B5F9
:1033500050F82140DCB1202383F31188D4F8942461
:103360001368527903EB8203DB689B695D6845B1A2
:1033700004216018FFF770FE294604F1140001F0E3
:1033800047FD2046FFF7BAFE002383F3118838BDBE
:103390007047000001F00AB9012303700023C0E95F
:1033A0000133C36183620362C36243620363704794
:1033B00038B50446202383F311880025C0E903555E
:1033C000C0E90555416001F001F90223237085F33E
:1033D000118838BD70B500EB810305465069DA608D
:1033E0000E46144618B110220021FEF7CBFBA0694F
:1033F00018B110220021FEF7C5FB31462846BDE872
:10340000704001F0ADB90000826802F001128260E4
:103410000022C0E90422826101F02EBAF0B400EB70
:1034200081044789E4680125A4698D403D434581B5
:1034300023600023A2606360F0BC01F049BA000081
:10344000F0B400EB81040789E468012564698D40CC
:103450003D43058123600023A2606360F0BC01F05E
:10346000C3BA000070B50223002504460370C0E90A
:103470000255C0E90455C564856180F8345001F0F7
:103480000BF963681B6823B129462046BDE87040EC
:10349000184770BD037880F85030052303704368E7
:1034A0001B6810B504460BB1042198470023A360A4
:1034B00010BD000090F85020436802701B680BB1EB
:1034C000052118477047000070B590F83430044665
:1034D00013B1002380F8343004F14402204601F097
:1034E000EDF963689B68B3B994F8443013F0600554
:1034F00035D00021204601F03FFC0021204601F09C
:1035000031FC63681B6813B10621204698470623E7
:1035100084F8343070BD204698470028E4D0B4F8D1
:103520004A30E26B9A4288BFE36394F94430E56B1A
:10353000002B4FF0200380F20381002D00F0F28079
:10354000092284F8342083F311880021D4E90E2362
:103550002046FFF775FF002383F31188DAE794F81C
:10356000452003F07F0343EA022340F202329342F4
:1035700000F0C58021D8B3F5807F48D00DD8012B4D
:103580003FD0022B00F09380002BB2D104F14C020B
:10359000A2630222E2632364C1E7B3F5817F00F0F6
:1035A0009B80B3F5407FA4D194F84630012BA0D185
:1035B000B4F84C3043F0020332E0B3F5006F4DD065
:1035C00017D8B3F5A06F31D0A3F5C063012B90D805
:1035D000636894F846205E6894F84710B4F8483061
:1035E0002046B047002884D04368A3630368E363A0
:1035F0001AE0B3F5106F36D040F6024293427FF4E2
:1036000078AF5C4BA3630223E3630023C3E794F822
:103610004630012B7FF46DAFB4F84C3023F0020339
:10362000C4E90E55A4F84C30256478E7B4F844306A
:10363000B3F5A06F0ED194F8463084F84E30204692
:1036400001F082F863681B6813B101212046984796
:10365000032323700023C4E90E339CE704F14F03D6
:10366000A3630123C3E72378042B10D1202383F322
:1036700011882046FFF7C8FE85F31188032163688F
:1036800084F84F5021701B680BB12046984794F87E
:103690004630002BDED084F84F300423237063685B
:1036A0001B68002BD6D0022120469847D2E794F819
:1036B00048301D0603F00F0120460AD501F0F0F84E
:1036C000012804D002287FF414AF2B4B9AE72B4B30
:1036D00098E701F0D7F8F3E794F84630002B7FF431
:1036E00008AF94F8483013F00F01B3D01A06204603
:1036F00002D501F055FBADE701F048FBAAE794F8CD
:103700004630002B7FF4F5AE94F8483013F00F01EB
:10371000A0D01B06204602D501F02EFB9AE701F04F
:1037200021FB97E7142284F8342083F311882B4679
:103730002A4629462046FFF771FE85F31188E9E6FF
:103740005DB1152284F8342083F311880021D4E977
:103750000E232046FFF762FEFDE60B2284F834209C
:1037600083F311882B462A4629462046FFF768FE38
:10377000E3E700BF545800084C58000850580008B0
:1037800038B590F834300446002B3ED0063BDAB210
:103790000F2A34D80F2B32D8DFE803F03731310845
:1037A000223231313131313131313737C56BB0F8F7
:1037B0004A309D4214D2C3681B8AB5FBF3F203FB67
:1037C00012556DB9202383F311882B462A462946CA
:1037D000FFF736FE85F311880A2384F834300EE0B3
:1037E000142384F83430202383F3118800231A46ED
:1037F00019462046FFF712FE002383F3118838BDD7
:10380000036C03B198470023E7E70021204601F04D
:10381000B3FA0021204601F0A5FA63681B6813B1D2
:103820000621204698470623D7E7000010B590F8F8
:103830003430142B044629D017D8062B05D001D8D4
:103840001BB110BD093B022BFBD80021204601F023
:1038500093FA0021204601F085FA63681B6813B1D2
:10386000062120469847062319E0152BE9D10B23A2
:1038700080F83430202383F3118800231A46194638
:10388000FFF7DEFD002383F31188DAE7C3689B6945
:103890005B68002BD5D1036C03B19847002384F8F3
:1038A0003430CEE7024B0022C3E900339A60704700
:1038B000F4350020002303748268054B1B68996867
:1038C0009142FBD25A6803604260106058607047B2
:1038D000F435002008B5202383F31188037C032BE3
:1038E00005D0042B0DD02BB983F3118808BD436993
:1038F00000221A604FF0FF334361FFF7DBFF002324
:10390000F2E7D0E9003213605A60F3E70023037452
:103910008268054B1B6899689142FBD85A6803601E
:103920004260106058607047F4350020054B1969FB
:103930000874186802681A605360186101230374E0
:10394000FCF766BEF435002030B54B1C0B4D87B03C
:10395000044610D02B690A4A01A800F025F9204638
:10396000FFF7E4FF049B13B101A800F059F92B699C
:10397000586907B030BDFFF7D9FFF8E7F4350020EC
:10398000D538000838B50C4D41612B6981689A68BB
:103990009142044603D8BDE83840FFF78BBF184674
:1039A000FFF7B4FF01232C61014623742046BDE8D4
:1039B0003840FCF72DBE00BFF4350020044B1A68D8
:1039C0001B6990689B68984294BF00200120704753
:1039D000F435002010B5084C236820691A6822606D
:1039E0005460012223611A74FFF790FF0146206999
:1039F000BDE81040FCF70CBEF435002008B5FFF719
:103A0000DDFF18B1BDE80840FFF7E4BF08BD0000C6
:103A1000FFF7E0BFFEE7000010B50C4CFFF742FFD8
:103A200000F0B4F80A498022204600F03BF8012358
:103A300044F8180C037400F0D3FC002383F31188BE
:103A400062B60448BDE8104000F04CB81C360020B7
:103A5000585800086858000800F01CB9EFF31180AE
:103A600020B9EFF30583202282F31188704700000C
:103A700010B530B9EFF30584C4F3080414B180F332
:103A8000118810BDFFF7BAFF84F31188F9E7000031
:103A9000034A516853685B1A9842FBD8704700BFCD
:103AA000001000E082600222028270478368A3F166
:103AB0007C0243F80C2C026943F83C2C426943F821
:103AC000382C074A43F81C2CC26843F8102C0222F9
:103AD00003F8082C002203F8072CA3F11800704704
:103AE0002906000810B5202383F31188FFF7DEFFB5
:103AF00000210446FFF746FF002383F31188204688
:103B000010BD0000024B1B6958610F20FFF70EBF6C
:103B1000F4350020202383F31188FFF7F3BF000062
:103B200008B50146202383F311880820FFF70CFF16
:103B3000002383F3118808BD49B1064B42681B6915
:103B400018605A60136043600420FFF7FDBE4FF019
:103B5000FF307047F43500200368984206D01A6899
:103B60000260506059611846FFF7A4BE704700001C
:103B700038B504460D462068844200D138BD03683C
:103B800023605C604561FFF795FEF4E7054B03F1A8
:103B90001402C3E905224FF0FF310022C3E90712E6
:103BA000704700BFF435002070B51C4EC0E90323F8
:103BB00005460C4601F0DCFA334653F8142F9A42BE
:103BC0000DD13062C5E901242A600A2C2CBF0019EE
:103BD0000A30C6E90555BDE8704001F0B7BA316A50
:103BE000431AE31838BF1C469368A34202D9081948
:103BF00001F0BAFA73699A6894420CD85A68AC60BA
:103C00002B606A6015609A685D60121B9A604FF0C5
:103C1000FF33F36170BD1B68A41AECE7F435002094
:103C200038B51B4C636998420DD0D0E9003213605F
:103C30005A6000228168C2609A680A449A604FF014
:103C4000FF33E36138BD2246036842F8143F002188
:103C500093425A60C16003D1BDE8384001F07EBA9A
:103C60009A688168256A0A449A6001F081FA63695A
:103C70009A68411B8A42E5D9AB181D1A092D206AA2
:103C800098BF01F10A02BDE83840104401F06CBA57
:103C9000F43500202DE9F041184C002704F11406FA
:103CA000656901F065FA236AAA68C11A8A4215D8C3
:103CB00013442362D5E9003213605A606369D5F872
:103CC0000C80EF60B34201D101F048FA87F311880C
:103CD0002869C047202383F31188E1E76169B14275
:103CE00009D013441B1ABDE8F0410A2B2CBFC018A1
:103CF0000A3001F039BABDE8F08100BFF435002088
:103D000000207047FEE70000704700004FF0FF30D2
:103D10007047000002290CD0032904D0012907486C
:103D200018BF00207047032A05D8054800EBC200E1
:103D30007047044870470020704700BF4C59000886
:103D4000302300200059000870B59AB00546084697
:103D500001A9144600F0C2F801A8FDF70BFF431CAF
:103D60005B00C5E900340022237003236370C6B2F0
:103D700001AB02341046D1B28E4204F1020401D8E4
:103D80001AB070BD13F8011B04F8021C04F8010CF2
:103D90000132F0E708B5202383F311880348FFF7C9
:103DA00079FA002383F3118808BD00BFB0370020E3
:103DB00090F8443003F01F02012A07D190F8452003
:103DC0000B2A03D10023C0E90E3315E003F0600392
:103DD000202B08D1B0F848302BB990F84520212A83
:103DE00003D81F2A04D8FFF737BA222AEBD0FAE704
:103DF000034A82630722C26303640120704700BF45
:103E00002823002007B5052917D8DFE801F0191687
:103E100003191920202383F31188104A01900121EE
:103E2000FFF7D8FA01980E4A0221FFF7D3FA0D489E
:103E3000FFF7FCF9002383F3118803B05DF804FB5E
:103E4000202383F311880748FFF7C6F9F2E7202300
:103E500083F311880348FFF7DDF9EBE7A05800086A
:103E6000C4580008B037002038B50C4D0C4C0D4933
:103E70002A4604F10800FFF767FF05F1CA0204F1C2
:103E800010000949FFF760FF05F5CA7204F1180038
:103E90000649BDE83840FFF757BF00BF783C002017
:103EA00030230020805800088A58000895580008E0
:103EB00070B5044608460D46FDF75CFEC6B22046C6
:103EC000013403780BB9184670BD32462946FDF718
:103ED0003DFE0028F3D10120F6E700002DE9F04770
:103EE00005460C46FDF746FE2B49C6B22846FFF7AD
:103EF000DFFF08B10B36F6B228492846FFF7D8FF96
:103F000008B11036F6B2632E0BD8DFF88C80DFF8DC
:103F10008C90234FDFF894A02E7846B92670BDE828
:103F2000F08729462046BDE8F04701F0E5BB252E85
:103F30002ED1072241462846FDF708FE70B9194BDD
:103F4000224603F1100153F8040B42F8040B8B4294
:103F5000F9D11B88138007351234DDE70822494662
:103F60002846FDF7F3FD98B90F4BA21C19780909F3
:103F70000232C95D02F8041C13F8011B01F00F01A5
:103F80005345C95D02F8031CF0D118340835C3E766
:103F900004F8016B0135BFE76C590008955800081B
:103FA0008759000874590008107AFF1F1C7AFF1FF8
:103FB000BFF34F8F024AD368DB03FCD4704700BFC6
:103FC000003C024008B5094B1B7873B9FFF7F0FFBE
:103FD000074B1A69002ABFBF064A5A6002F18832AD
:103FE0005A601A6822F480621A6008BDD63E00202A
:103FF000003C02402301674508B50B4B1B7893B981
:10400000FFF7D6FF094B1A6942F000421A611A689D
:1040100042F480521A601A6822F480521A601A68B8
:1040200042F480621A6008BDD63E0020003C024087
:104030000B28F0B516D80C4C0C4923787BB90C4DE5
:104040000E460C234FF0006255F8047B46F8042B13
:10405000013B13F0FF033A44F6D10123237051F8DA
:104060002000F0BD0020FCE7083F0020D83E0020E3
:1040700098590008014B53F82000704798590008E0
:104080000C2070470B2810B5044601D9002010BD44
:10409000FFF7CEFF064B53F824301844C21A0BB971
:1040A0000120F4E712680132F0D1043BF6E700BFCB
:1040B000985900080B2810B5044621D8FFF778FF5F
:1040C000FFF780FF0F4AF323D360C300DBB243F452
:1040D000007343F002031361136943F480331361E7
:1040E000FFF766FFFFF7A4FF074B53F8241000F01B
:1040F00029F9FFF781FF2046BDE81040FFF7C2BF56
:10410000002010BD003C024098590008F8B512F09C
:104110000103144642D18218B2F1016F57D82D4BDA
:104120001B6813F0010352D02B4DFFF74BFFF32315
:10413000EB60FFF73DFF40F20127032C15D824F078
:1041400001046618244C401A40F20117B142236959
:1041500000EB010524D123F001032361FFF74CFF9D
:104160000120F8BD043C0430E7E78307E7D12B6961
:1041700023F440732B612B693B432B6151F8046B93
:104180000660BFF34F8FFFF713FF03689E42E9D02D
:104190002B6923F001032B61FFF72EFF0020E0E7DE
:1041A00023F44073236123693B4323610B882B80F5
:1041B000BFF34F8FFFF7FCFE2D8831F8023BADB205
:1041C000AB42C3D0236923F001032361E4E718461F
:1041D000C7E700BF00380240003C0240084908B56C
:1041E0000B7828B11BB9FFF7EDFE01230B7008BD5A
:1041F000002BFCD0BDE808400870FFF7FDBE00BFF3
:10420000D63E002070B582B0FFF728FC0E4E054662
:1042100000F0AEFF3268904237BF0C4A0B4951683C
:1042200014682EBFD1E900410131516004190346E1
:1042300041F10001284601913360FFF719FC019913
:10424000204602B070BD00BF0C3F0020103F002090
:1042500070B582B0FFF702FC104E054600F088FFF3
:104260003268904237BF0E4A0D49516814682EBF1C
:10427000D1E9004101315160041941F100010346C7
:10428000284601913360FFF7F3FB01994FF47A72EE
:1042900000232046FBF7A4FF02B070BD0C3F0020B6
:1042A000103F002010B50244064BD2B2904200D11C
:1042B00010BD441C00B253F8200041F8040BE0B2DA
:1042C000F4E700BF502800400F4B30B51C6F2404AA
:1042D00007D41C6F44F400741C671C6F44F4004442
:1042E0001C670A4C236843F4807323600244084B24
:1042F000D2B2904200D130BD441C00B251F8045BF0
:1043000043F82050E0B2F4E700380240007000406B
:104310005028004007B5012201A90020FFF7C2FF85
:10432000019803B05DF804FB13B50446FFF7F2FFF4
:10433000A04205D0012201A900200194FFF7C4FF8B
:1043400002B010BD70470000074B45F255521A608D
:1043500002225A6040F6FF729A604CF6CC421A6014
:10436000024B01221A70704700300040193F0020B4
:10437000034B1B781BB1034B4AF6AA221A60704705
:10438000193F002000300040044BD3F874389B00E4
:1043900042BF034B01221A70704700BF0030024039
:1043A000183F0020024B4FF08072C3F8742870470A
:1043B00000300240014B1878704700BF183F0020C2
:1043C000EFF3098305494A6B22F001024A6368331F
:1043D00083F30988002383F31188704700EF00E01E
:1043E000202080F3118862B60C4B0D4AD96821F465
:1043F000E0610904090C0A43DA60D3F8FC2009499A
:1044000042F08072C3F8FC200A6842F001020A60A0
:104410001022DA7783F82200704700BF00ED00E039
:104420000003FA05001000E010B5202383F3118883
:104430000E4B5B6813F4006314D0F1EE103AEFF307
:104440000984683C4FF08073E361094BDB6B2366A2
:1044500084F30988FFF7B2FA10B1064BA36110BDCF
:10446000054BFBE783F31188F9E700BF00ED00E09F
:1044700000EF00E03B0600083E0600087047000021
:10448000FEE700000A4B0B480B4A90420BD30B4B44
:10449000DA1C121AC11E22F003028B4238BF00221E
:1044A0000021FDF76FBB53F8041B40F8041BECE739
:1044B000505B0008144000201440002014400020ED
:1044C0007047000070B5D0E915439E6800224FF098
:1044D000FF3504EB42135101D3F800090028BEBF99
:1044E000D3F8000940F08040C3F80009D3F8000B6E
:1044F0000028BEBFD3F8000B40F08040C3F8000B8B
:10450000013263189642C3F80859C3F8085BE0D239
:104510004FF00113C4F81C3870BD00001D4B03EBB5
:1045200080022DE9F043D2F80CC05D6DDCF8142058
:10453000461CD2F800E005EB063605EB4018516842
:1045400071450AD3D5F83438012202FA00F023EA83
:104550000000C5F83408BDE8F083BCF81040AEEBAD
:104560000103A34228BF2346D8F81849A4B2B3EBED
:10457000840FF0D89468A4F1040959F8047F3760D7
:10458000A4EB09071F44042FF7D81C440B44946084
:104590005360D4E71C3F0020890141F020010161F4
:1045A00003699B06FCD41220FFF772BA10B5054CC4
:1045B0002046FEF7F1FE4FF0A0436365024BA36572
:1045C00010BD00BF1C3F0020EC59000870B50378F7
:1045D000012B054650D12A4B446D98421BD1294BE3
:1045E0005A6B42F080025A635A6D42F080025A655B
:1045F0005A6D5A6942F080025A615A6922F080026B
:104600005A610E2143205B69FEF79CFC1E4BE36060
:104610001E4BC4F800380023C4F8003EC0232360BA
:104620006E6D4FF40413A3633369002BFCDA01238E
:1046300033610C20FFF72CFA3369DB07FCD412201E
:10464000FFF726FA3369002BFCDA0026A66028461D
:10465000FFF738FF6B68C4F81068DB68C4F81468AB
:10466000C4F81C684BB90A4BA3614FF0FF33636178
:10467000A36843F00103A36070BD064BF4E700BFDD
:104680001C3F00200038024040140040030020027C
:10469000003C30C0083C30C0F8B5446D05460021F0
:1046A0002046FFF779FFA96D00234FF001128F68B4
:1046B000C4F834384FF00066C4F81C284FF0FF30BF
:1046C00004EB431201339F42C2F80069C2F8006B49
:1046D000C2F80809C2F8080BF2D20B686A6DEB65E4
:1046E000636210231361166916F01006FBD11220C5
:1046F000FFF7CEF9D4F8003823F4FE63C4F800388D
:10470000A36943F4402343F01003A3610923C4F8D1
:104710001038C4F814380A4BEB604FF0C043C4F8AB
:10472000103B084BC4F8003BC4F81069C4F80039CA
:10473000EB6D03F1100243F48013EA65A362F8BD48
:10474000C859000840800010426D90F84E10D2F811
:10475000003823F4FE6343EA0113C2F800387047BF
:104760002DE9F84300EB8103456DDA68166806F021
:104770000306731E022B05EB41130C4680460FFA0D
:1047800081F94FEA41104FF00001C3F8101B4FF0C0
:10479000010104F1100398BFB60401FA03F3916913
:1047A0008EBF334E06F1805606F5004600293AD0FA
:1047B000578A04F15801490137436F50D5F81C1846
:1047C0000B43C5F81C382B180021C3F81019536986
:1047D0000127611EA7409BB3138A928B9B08012A75
:1047E00088BF5343D8F85C20981842EA034301F18C
:1047F000400205EB8202C8F85C002146536028465F
:10480000FFF7CAFE08EB8900C3681B8A43EA84539A
:10481000483464011E432E51D5F81C381F43C5F897
:104820001C78BDE8F88305EB4917D7F8001B21F485
:104830000041C7F8001BD5F81C1821EA0303C0E7A4
:1048400004F13F0305EB83030A4A5A6028462146D8
:10485000FFF7A2FE05EB4910D0F8003923F400431E
:10486000C0F80039D5F81C3823EA0707D7E700BF9E
:104870000080001000040002826D1268C265FFF71C
:1048800021BE00005831436D49015B5813F40040CC
:1048900004D013F4001F0CBF022001207047000059
:1048A0004831436D49015B5813F4004004D013F4C0
:1048B000001F0CBF022001207047000000EB8101A7
:1048C000CB68196A0B6813604B685360704700002F
:1048D00000EB810330B5DD68AA691368D36019B9AC
:1048E000402B84BF402313606B8A1468426D1C44C4
:1048F000013CB4FBF3F46343033323F0030302EB03
:10490000411043EAC44343F0C043C0F8103B2B6856
:1049100003F00303012B09B20ED1D2F8083802EBE1
:10492000411013F4807FD0F8003B14BF43F0805354
:1049300043F00053C0F8003B02EB4112D2F8003BB9
:1049400043F00443C2F8003B30BD00002DE9F041C4
:10495000244D6E6D06EB40130446D3F8087BC3F874
:10496000087B38070AD5D6F81438190706D505EBA1
:1049700084032146DB6828465B689847FA071FD501
:10498000D6F81438DB071BD505EB8403D968CCB9FE
:104990008B69488A5A68B2FBF0F600FB16228AB986
:1049A0001868DA6890420DD2121AC3E90024202355
:1049B00083F311880B482146FFF78AFF84F311889F
:1049C000BDE8F081012303FA04F26B8923EA0203B4
:1049D0006B81CB68002BF3D021460248BDE8F04143
:1049E000184700BF1C3F002000EB810370B5DD6855
:1049F000436D6C692668E6604A0156BB1A444FF461
:104A00000020C2F810092A6802F00302012A0AB243
:104A10000ED1D3F8080803EB421410F4807FD4F8C9
:104A2000000914BF40F0805040F00050C4F8000965
:104A300003EB4212D2F8000940F00440C2F800092A
:104A4000D3F83408012202FA01F10143C3F8341803
:104A500070BD19B9402E84BF4020206020682E8A86
:104A60008419013CB4FBF6F440EAC44040F0005025
:104A70001A44C6E7F8B504461E48456D05EB4413D5
:104A8000D3F80869C3F80869F10717D5D5F81038C5
:104A9000DA0713D500EB8403D9684B691F68DA681D
:104AA000974218D2D21B00271A605F60202383F33D
:104AB00011882146FFF798FF87F31188330617D531
:104AC000D5F834280123A340134211D02046BDE875
:104AD000F840FFF723BD012303FA04F2038923EA18
:104AE000020303818B68002BE8D021469847E5E755
:104AF000F8BD00BF1C3F00202DE9F74F984C666DB4
:104B00007569B3691D4015F48058756107D020465A
:104B1000FEF7A8FC03B0BDE8F04FFFF785BC002D01
:104B200012DAD6F8003E8E489F071EBFD6F8003E28
:104B300023F00303C6F8003ED6F8043823F001033F
:104B4000C6F80438FEF7B6FC280505D58448FFF7FB
:104B5000B9FC8348FEF79EFCA9040CD5D6F80838AA
:104B600013F0060FF36823F470530CBF43F4105393
:104B700043F4A053F3602A0704D56368DB680BB1E4
:104B800077489847EB0274D4AF0227D5D4F85490F5
:104B9000DFF8CCB100274FF0010A09EB4712D2F839
:104BA000003B03F44023B3F5802F11D1D2F8003B32
:104BB000002B0DDA62890AFA07F322EA0303638104
:104BC00004EB8703DB68DB6813B139465846984726
:104BD000A36D01379B68FFB29F42DED9E80617D567
:104BE000676D3A6AC2F30A1002F00F0302F4F01282
:104BF000B2F5802F00F08880B2F5402F08D104EB89
:104C000083030022DB681B6A07F5805790426DD151
:104C10002903D6F8184813D5E20302D50020FFF780
:104C200095FEA30302D50120FFF790FE670302D58E
:104C30000220FFF78BFE260302D50320FFF786FE36
:104C40006D037FF567AFE00702D50020FFF712FF85
:104C5000A10702D50120FFF70DFF620702D5022050
:104C6000FFF708FF23077FF555AF0320FFF702FF8B
:104C700050E7636DDFF8E8B0019300274FF0010AB9
:104C8000A36D9B685FFA87F999453FF67DAF019B5D
:104C900003EB4913D3F8002902F44022B2F5802F28
:104CA00022D1D3F80029002A1EDAD3F8002942F0D5
:104CB0009042C3F80029D3F80029002AFBDB606D7D
:104CC0004946FFF769FC22890AFA09F322EA03033D
:104CD000238104EB8903DB689B6813B1494658467E
:104CE00098474846FFF71AFC0137C9E7910708BF04
:104CF000D7F80080072A98BF03F8018B02F1010260
:104D000098BF4FEA182881E7023304EB830207F5C6
:104D100080575268D2F818C0DCF80820DCE9001C83
:104D2000A1EB0C0C002188420AD104EB83046368D8
:104D30009B699A6802449A605A6802445A6067E71D
:104D400011F0030F08BFD7F800808C4588BF02F828
:104D5000018B01F1010188BF4FEA1828E3E700BF8A
:104D60001C3F0020436D03EB4111D1F8003B43F49D
:104D70000013C1F8003B7047436D03EB4111D1F8BC
:104D8000003943F40013C1F800397047436D03EB59
:104D90004111D1F8003B23F40013C1F8003B7047E8
:104DA000436D03EB4111D1F8003923F40013C1F82E
:104DB0000039704730B5039C0172043304FB0325AE
:104DC000C0E90653049B03630021059BC160C0E951
:104DD0000000C0E90422C0E90842C0E90A114363A7
:104DE00030BD0000416A0022C0E90411C0E90A2276
:104DF000C2606FF00101FEF7BBBE0000D0E90432D3
:104E0000934201D1C2680AB9181D7047002070474B
:104E100003691960C2680132C260C26913448269C1
:104E20000361934224BF436A03610021FEF794BEED
:104E300038B504460D46E3683BB16269131D12683C
:104E4000A3621344E362002007E0237A33B92946C2
:104E50002046FEF771FE0028EDDA38BD6FF0010044
:104E6000FBE70000C368C269013BC36043691344A8
:104E700082694361934224BF436A43610023836292
:104E8000036B03B11847704770B52023044683F3C2
:104E90001188866A3EB9FFF7CBFF054618B186F345
:104EA0001188284670BDA36AE26A13F8015BA36209
:104EB000934202D32046FFF7D5FF002383F31188E6
:104EC000EFE700002DE9F84F04460E4617469846D6
:104ED0004FF0200989F311880025AA46D4F828B09C
:104EE000BBF1000F09D141462046FFF7A1FF20B1D9
:104EF0008BF311882846BDE8F88FD4E90A12A7EB96
:104F0000050B521A934528BF9346BBF1400F1BD99E
:104F1000334601F1400251F8040B43F8040B91426F
:104F2000F9D1A36A40334036A3624035D4E90A235D
:104F30009A4202D32046FFF795FF8AF31188BD42BB
:104F4000D8D289F31188C9E730465A46FCF7F4FDF8
:104F5000A36A5B445E44A3625D44E7E710B5029C2C
:104F60000172043304FB0321C0E906130023C0E9E6
:104F70000A33039B0363049BC460C0E90000C0E9DB
:104F80000422C0E90842436310BD0000026AC26007
:104F9000426AC0E904220022C0E90A226FF001013E
:104FA000FEF7E6BDD0E904239A4201D1C26822B9D6
:104FB000184650F8043B0B60704700207047000013
:104FC000C368C2690133C3604369134482694361A2
:104FD000934224BF436A43610021FEF7BDBD000038
:104FE00038B504460D46E3683BB123691A1DA26239
:104FF000E2691344E362002007E0237A33B92946CB
:105000002046FEF799FD0028EDDA38BD6FF001006B
:10501000FBE7000003691960C268013AC260C26917
:10502000134482690361934224BF436A03610023EE
:105030008362036B03B118477047000070B52023EB
:105040000D460446114683F31188866A2EB9FFF790
:10505000C7FF10B186F3118870BDA36A1D70A36AE3
:10506000E26A01339342A36204D3E1692046043922
:10507000FFF7D0FF002080F31188EDE72DE9F84F0E
:1050800004460D46904699464FF0200A8AF311884F
:105090000026B346A76A4FB949462046FFF7A0FF4E
:1050A00020B187F311883046BDE8F88FD4E90A07AC
:1050B0003A1AA8EB0607974228BF1746402F1BD97C
:1050C00005F1400355F8042B40F8042B9D42F9D11B
:1050D000A36A4033A3624036D4E90A239A4204D338
:1050E000E16920460439FFF795FF8BF311884645A7
:1050F000D9D28AF31188CDE729463A46FCF71CFD40
:10510000A36A3B443D44A3623E44E5E7D0E904235F
:105110009A4217D1C3689BB1836A8BB1043B9B1A37
:105120000ED01360C368013BC360C3691A4483692E
:1051300002619A4224BF436A036100238362012310
:10514000184670470023FBE700F088B84FF0804313
:10515000002258631A610222DA6070474FF08043E0
:105160000022DA60704700004FF0804358637047B8
:105170004FF08043586A70474B6843608B68836088
:10518000CB68C3600B6943614B6903628B694362FF
:105190000B6803607047000008B5264B26481A6963
:1051A00040F2FF110A431A611A6922F4FF7222F0D9
:1051B00001021A611A691A6B0A431A631A6D0A43CB
:1051C0001A651E4A1B6D1146FFF7D6FF02F11C013E
:1051D00000F58060FFF7D0FF02F1380100F5806034
:1051E000FFF7CAFF02F1540100F58060FFF7C4FF2A
:1051F00002F1700100F58060FFF7BEFF02F18C0143
:1052000000F58060FFF7B8FF02F1A80100F58060AB
:10521000FFF7B2FF02F1C40100F58060FFF7ACFFB9
:1052200002F1E00100F58060FFF7A6FFBDE808404D
:1052300000F09AB80038024000000240F859000817
:1052400008B500F007FAFEF7E7FBFFF79DF8BDE8A9
:105250000840FEF709BE000070470000104B1A6CB2
:1052600042F001021A641A6E42F001021A660D4AF7
:105270001B6E936843F0010393604FF08043532209
:105280009A624FF0FF32DA6200229A615A63DA6062
:105290005A6001225A6108211A601C20FDF752BE93
:1052A00000380240002004E04FF0804208B5116948
:1052B000D3680B40D9B2C9439B07116107D520239E
:1052C00083F31188FEF7C8FB002383F3118808BD20
:1052D00008B5FFF7E9FFBDE80840FFF7A5B80000F3
:1052E0001F4B1A696FEAC2526FEAD2521A611A69E9
:1052F000C2F308021A614FF0FF301A695A69586107
:1053000000215A6959615A691A6A62F080521A6218
:105310001A6A02F080521A621A6A5A6A58625A6A03
:1053200059625A6A1A6C42F080521A641A6E42F03C
:1053300080521A661A6E0B4A106840F48070106032
:10534000186F00F44070B0F5007F1EBF4FF480303E
:1053500018671967536823F40073536000F05AB953
:105360000038024000700040334B4FF080521A6406
:10537000324A4FF4404111601A6842F001021A604B
:105380001A689107FCD59A6822F003029A602A4BAA
:105390009A6812F00C02FBD1196801F0F90119604A
:1053A0009A601A6842F480321A601A689203FCD537
:1053B0005A6F42F001025A671F4B5A6F9007FCD593
:1053C0001F4A5A601A6842F080721A601B4A53687A
:1053D0005904FCD5184B1A689201FCD5194A9A60F9
:1053E000194B1A68194B9A42194B21D1194A116865
:1053F000194A91421CD140F205121A60144A1368EE
:1054000003F00F03052BFAD10B4B9A6842F002020E
:105410009A609A6802F00C02082AFAD15A6C42F497
:1054200080425A645A6E42F480425A665B6E7047FC
:1054300040F20572E1E700BF003802400070004012
:105440000854400700948838002004E011640020CC
:10545000003C024000ED00E041C20F41084A08B59F
:10546000516913680B4003F00103536123B1054AEE
:1054700013680BB150689847BDE80840FEF7D4BFE9
:10548000003C0140943F0020084A08B55169136868
:105490000B4003F00203536123B1054A93680BB13B
:1054A000D0689847BDE80840FEF7BEBF003C014009
:1054B000943F0020084A08B5516913680B4003F077
:1054C0000403536123B1054A13690BB1506998472E
:1054D000BDE80840FEF7A8BF003C0140943F002013
:1054E000084A08B5516913680B4003F0080353617B
:1054F00023B1054A93690BB1D0699847BDE80840CC
:10550000FEF792BF003C0140943F0020084A08B5D6
:10551000516913680B4003F01003536123B1054A2E
:10552000136A0BB1506A9847BDE80840FEF77CBF8C
:10553000003C0140943F0020174B10B55A691C688D
:10554000144004F478725A61A30604D5134A936A8E
:105550000BB1D06A9847600604D5104A136B0BB1A3
:10556000506B9847210604D50C4A936B0BB1D06B56
:105570009847E20504D5094A136C0BB1506C984763
:10558000A30504D5054A936C0BB1D06C9847BDE8D0
:105590001040FEF749BF00BF003C0140943F00208F
:1055A0001A4B10B55A691C68144004F47C425A61C5
:1055B000620504D5164A136D0BB1506D984723054B
:1055C00004D5134A936D0BB1D06D9847E00404D510
:1055D0000F4A136E0BB1506E9847A10404D50C4AC4
:1055E000936E0BB1D06E9847620404D5084A136FCE
:1055F0000BB1506F9847230404D5054A936F0BB144
:10560000D06F9847BDE81040FEF70EBF003C014048
:10561000943F0020062108B50846FDF793FC0621BB
:105620000720FDF78FFC06210820FDF78BFC0621E3
:105630000920FDF787FC06210A20FDF783FC0621DF
:105640001720FDF77FFCBDE8084006212820FDF764
:1056500079BC000008B5FFF743FE00F00DF8FDF738
:1056600087FCFDF797FEFDF76FFDFFF7F5FDBDE841
:105670000840FFF769BD00000023054A19460133C1
:10568000102BC2E9001102F10802F8D1704700BFE7
:10569000943F002010B501390244904201D100200E
:1056A00005E0037811F8014FA34201D0181B10BD8B
:1056B0000130F2E72DE9F041A3B1C91A177801448E
:1056C000044603F1FF3C8C42204601D9002009E04A
:1056D0000578BD4204F10104F5D10CEB0405D618A0
:1056E000A54201D1BDE8F08115F8018D16F801ED54
:1056F000F045F5D0E7E70000034611F8012B03F869
:10570000012B002AF9D170476F72672E61726475A0
:1057100070696C6F742E663430355F4D6174656BE3
:105720004169727370656564000000004E6F20610E
:105730007070207369670A00426164206677206C8C
:10574000656E6774682025750A0042616420626F87
:105750006172645F69642025752073686F756C647D
:105760002062652025750A00426164206677206406
:10577000657363726970746F72206C656E677468AC
:105780002025750A004261642061707020435243F5
:10579000203078253038783A307825303878203005
:1057A00078253038783A3078253038780A00476FD5
:1057B0006F64206669726D776172650A0040A2E4C9
:1057C000F16468910600000053544D3332463F3F68
:1057D0003F00000053544D33324634307800535468
:1057E0004D3332463432780053544D3332463434DC
:1057F0003658580000000000C85700083F0000005D
:1058000013040000D45700083F00000019040000F2
:10581000DE5700083F00000021040000E8570008A0
:105820003F00000000000000C5300008B130000853
:10583000ED300008D9300008E5300008D13000080C
:10584000BD300008A9300008F93000080000000051
:1058500001000000000000006D61696E00000000A2
:1058600069646C650000000060580008383600204C
:10587000B037002001000000153A000800000000C9
:105880004172647550696C6F740025424F415244F7
:10589000252D424C002553455249414C250000001E
:1058A0000200000000000000E13200084D33000853
:1058B00040004000483C0020583C0020020000000E
:1058C0000000000003000000000000009133000809
:1058D0000000000010000000683C002000000000F4
:1058E00001000000000000001C3F00200101020038
:1058F000053E0008153D0008B13D0008953D000833
:10590000430000000859000809024300020100C0DA
:105910003209040000010202010005240010010503
:105920002401000104240202052406000107058267
:10593000030800FF09040100020A00000007050136
:105940000240000007058102400000001200000034
:105950005459000812011001020000400912415779
:1059600000020102030100000403090425424F4123
:1059700052442500663430352D4D6174656B4169A4
:1059800072737065656400303132333435363738C0
:1059900039414243444546000040000000400000B9
:1059A0000040000000400000000001000000020074
:1059B00000000200000002000000020000000200DF
:1059C000000002000000020000000000C9340008CE
:1059D000813700082D380008400040007C3F00203F
:1059E0007C3F0020010000008C3F00208000000070
:1059F0004001000003000000AA01A81200000000FE
:105A0000AAAAAAAA55011400FFBF000088770000C7
:105A100070A70A0000000A0100000000AAAAAAAAB2
:105A200000000001FFFF00000000000099000000DE
:105A30000000A01600000000AAAAAAA600005011AB
:105A4000FFDF0000000000000077080020000000D9
:105A500000000000AAAAAAAA10000000FFFF000090
:105A6000000800000000000000000000000000002E
:105A7000AAAAAAAA00000000FFFF00000000000080
:105A8000000000000000000000000000AAAAAAAA6E
:105A900000000000FFFF0000000000000000000008
:105AA0000000000000000000AAAAAAAA000000004E
:105AB000FFFF0000000000000000000000000000E8
:105AC000000000000A0000000000000003000000C9
:105AD00000000000000000000000000000000000C6
:105AE00000000000000000000000000000000000B6
:105AF000000000001CA7FF7F010000000000000064
:105B0000F60300000000000000000F00000000008D
:105B10006400000000000000FE2A0100D204000022
:105B2000FF0096000000000800960000000008003A
:105B30000400000068590008000000000000000098
:105B40000000000000000000000000000000000055
:00000001FF
